:10000000A0220020811900007D1900007D19000048
:1000100000000000000000000000000000000000E0
:100020000000000000000000000000007D1900003A
:1000300000000000000000007D1900007D19000094
:100040007D1900007D1900007D1900007D19000058
:100050007D1900007D190000790400007D19000061
:100060007D190000AD120000BD120000CD1200008D
:10007000DD120000ED120000FD1200007D190000ED
:100080007D1900007D1900007D1900007D19000018
:100090007D1900007D1900007D1900007D19000008
:1000A0007D1900007D1900007D1900007D190000F8
:1000B0000000000010B5064C2378002B07D1054B3B
:1000C000002B02D0044800E000BF0123237010BDC4
:1000D0008000002000000000545B0000084B10B5B9
:1000E000002B03D00749084800E000BF0748036819
:1000F000002B00D110BD064B002BFBD09847F9E731
:100100000000000084000020545B0000545B0000ED
:100110000000000030B597B002AD040050220A493B
:1001200028000A4B9847132C0BD80023A40001A9E0
:1001300060594B70CB708B7001330B70C0B2044BA5
:10014000984717B030BDC046F05800001548000071
:1001500021190000C0225201C281020000232A326C
:10016000037043704380037103760362C36183604D
:100170000373037443748374C37403751370421D53
:1001800043758375D377C3840385C37526322C30BA
:1001900013700370704700008023F0B51400AC4A60
:1001A00001600700106A5B02034313620B7887B09B
:1001B0000520DB0700D5E7E00B7817309B0700D55B
:1001C000E2E063783B71002B04D1A24A0433116C46
:1001D0000B431364237805A90B701E209E4B3D68CA
:1001E00098479E4B1E20984723002C3302931B7880
:1001F000227B0192002B33D022002B321678019AF9
:100200009619F6B29B19DBB20393019BF01A039B7C
:10021000C0B2B3421BD8E089914B9847637D9B00E5
:10022000DBB22B70A37D6278DB011343DBB26B7012
:100230002379302B00D1B4E018D8102B00D1ADE0D9
:10024000202B00D1ADE0002B1AD11A00A7E00F231C
:100250001840237B0136C018814B9847F6B2D4E78B
:1002600001987F4EB047E089B047D7E7322B09D0DD
:1002700000D298E0332B00D18CE0342B00D185E004
:10028000172081E00422102302217020090101407F
:100290000A43AA70E27D3F2AF2D8EA7039684A7EA2
:1002A00052B2002AFBDB6188E27C0A43611DC87FF1
:1002B000C0000243207D80000243A07C4000024336
:1002C0001A43AA80227E9446002A07D0102B00D120
:1002D000AFE000D969E0002B00D19BE03868437E95
:1002E0005BB2002BFBDB63462B723A68537E5BB23A
:1002F000002BFBDBA38BAB833A68537E5BB2002BF6
:10030000FBDB238C2B84029B1A78002A03D0013A52
:10031000D2B20F2AB4D823002B3318780F28AFD8C5
:100320003E68737E5BB2002BFBDB267BE389000516
:100330003343A66812043343034313432B61230062
:100340002A331B782B750F23AB75CB7F002B0CD07A
:10035000E38C44498B4293D8AB848023228D1B01CC
:10036000D3189BB28B428BD8EA84E0223E4B00200C
:100370001968D2004B0119001A403C4B1B68DB0E78
:100380000B43DBB213432B8507B0F0BD617C227CAD
:1003900010237AE706221023012176E708220021A4
:1003A00073E70022FBE70222F5E7202B18D0302B61
:1003B00000D093E7E37CE069002B09D00300803391
:1003C000FF2B00D95CE7236A8033FF2B00D957E766
:1003D000FF2800DD54E7236AFF2B00DD50E77DE7AF
:1003E000E07CE669224B00280CD080208000301889
:1003F000984200D944E78022206A9200101898425F
:1004000000D93DE79E4200DD3AE7226A9A4200DDCC
:1004100036E763E7E07CE669124B0028F2D08022E1
:100420001201B018984200D92AE78020226A000100
:10043000E4E7E07CE6690F4B0028E3D0802212025B
:10044000B018984200D91BE78020226A0002D5E745
:1004500000040040000800404D180000C5170000CF
:1004600015010000FF0F0000246080002060800064
:10047000FF030000FFFF000070B5204B98470F22DC
:100480001F4B20491B8C204C13409B0058581F4D7C
:10049000037813401E4A137001781E4A090164183C
:1004A0006918137864884988DBB2611A41611C00BD
:1004B00001210C400CD0102311704374037C0B42BB
:1004C00003D04368002B00D09847134B984770BD6A
:1004D00002210B4206D01170037C44740B42F4D00D
:1004E0008368EFE704210B42EFD0062311704374B9
:1004F000037C0B42E9D0C368E4E7C04679130000EF
:10050000004800419C000020E0010020B0000020D5
:100510003F4800414E480041AD1300000023032234
:10052000037043708270C37003717047F8B53F4B1E
:1005300005000E0098473E4F3B78002B16D1202235
:100540003C4B59690A435A611022D9690A43022176
:10055000DA61394B1A888A431A80012237491A8096
:10056000596337499963374919803A702F4B984737
:10057000002401237A681A424CD1A3407A681343BD
:100580007B603B7A013B3B7201272F4B9847002F42
:1005900047D02E4B02212C701C7001242C4B264F6F
:1005A0001A788A431A701C70204B98470F222B78B8
:1005B000FC211340254A890113702A783B69944035
:1005C0006022A3433B6133785B01134072781202CF
:1005D0000A40C0211343B278090492050A4013432C
:1005E000F278002A04D007210A4001310A4313435C
:1005F0003279002A01D01022134300247B64124B6D
:1006000098472B78134A9B009D50AC610E4B98473E
:100610002000F8BD0134E4B25208052CABD100270C
:10062000B3E7094B98471420F3E7C046791300005D
:10063000000000200004004000480041E0010020CC
:10064000B0000020020F0000AD1300003F48004141
:10065000404800419C00002070B50500184B9847A9
:100660006C7C184EE4B2052C02D1B047200070BD5E
:10067000AB695B88002B02D1B0471720F7E7402217
:10068000114B1A602B78313A1340104A13702B78B3
:100690000F4AD35C072213400E4A137005232878B3
:1006A0006B740D4B0001C018A96910220B4B9847C1
:1006B00002230B4A11780B431370B0470020D6E792
:1006C00079130000AD13000000E100E03F48004155
:1006D000000100204D480041E001002015480000C5
:1006E0004048004170B50124032603880A78A343DB
:1006F0002240134303804A7806253240A2400388F3
:10070000AB43134303808B7818223340B3400588F2
:1007100095431D430580CA780388184D3240120264
:100720002B40134303800A790388154D224092021F
:100730002B40134303804A790388124D22402B40FB
:10074000D202134303808A79038822400E4C12039D
:100750002340134303800723CA791A4003885203B6
:10076000DB04DB0C134303800B894380CB684360BD
:100770000B6983604B69C36070BDC046FFFCFFFF1F
:10078000FFFBFFFFFFF7FFFFFFEFFFFF0200437CD0
:100790000520834204D09369002B03D11800916196
:1007A0007047DB68D8680028FBD1D960F8E7000003
:1007B000F0B5002489B0009201933F230026002762
:1007C0002500069007910393039A134B0120002103
:1007D0009847B6197F41069B079A03400A40049642
:1007E0000597134303D0012333431E00059F019B4C
:1007F000BB4209D802D1009BB34205D8009A019BA5
:10080000B61A9F4104430D43039B5A1E0392DBD249
:100810002000290009B0F0BD7522000010B549087C
:10082000040000234020A14201D210BD0300581C47
:10083000091B80B28C42F9D94020FF2BF5D81380D8
:100840000020F2E7F0B585B01E000AAB0D00197864
:1008500003004B4303924027AB4217D8002E18D118
:100860000200330008001B4C3100A0472A000100A1
:100870003300194C3000A04700220123121A8B418B
:10088000140C180404430027039B1C80380005B097
:10089000F0BD0024012EF6D10A00230021000D4EE8
:1008A000B047009001910B000200210028000A4C83
:1008B000A047802306009B019842E7D8009A019B3D
:1008C000690FE800A047F400041BE4B2640334435A
:1008D000D9E7C04609230000B107000037B50D4C29
:1008E00005002378002B01D000290CD001A913208A
:1008F000094B0D7098471320084B9847012300209F
:10090000657023703EBD63780800AB42FAD01D20AD
:10091000F8E7C046050100204D180000C51700008B
:10092000394A030000B50800934233D007D8374A4C
:10093000934214D0364A93421FD0002317E0354A21
:1009400093423AD0344A934244D0344A9342F4D149
:10095000002303290BD801F0F7FB502A2C2E00238B
:10096000032904D801F0F0FB430205072C4B1800C3
:1009700000BD2C4BFBE72C4BF9E700230329F6D8ED
:1009800001F0E2FB37020406284BF0E7284BEEE7C4
:10099000284BECE700230329E9D801F0D5FB2C0212
:1009A0000406254BE3E7254BE1E7254BDFE7254B25
:1009B000DDE7254BDBE7254BD9E700230329D6D814
:1009C00001F0C2FB1D020406214BD0E7214BCEE70C
:1009D000214BCCE700230329C9D801F0B5FB120253
:1009E00004061E4BC3E71E4BC1E71E4BBFE71E4B61
:1009F000BDE70323BBE71D4BB9E71D4BB7E71D4B15
:100A0000B5E71D4BB3E7C0460010004200080042A6
:100A1000000C004200180042001C0042001400427A
:100A200003000500030006000300070003000100A7
:100A300003001E0003001F000300090003000A005A
:100A400003000B0003001100030012000300130059
:100A500003000D0003000E0003000F000300170049
:100A6000030018000300190003000400030008003D
:100A70000300100003000C000300160070B586B0E0
:100A80006946094B6A4670CB70C170CB70C10023B8
:100A900099005158814202D1D8B206B070BD0133DD
:100AA000062BF5D10020F8E74059000070B50E0084
:100AB00014001500002808D0012040420CE0074B2C
:100AC000013D1868064B1B689847611B7118002D83
:100AD000F5DCE043C017204070BDC046380200205E
:100AE00030020020013870B50E0002280DD80C002D
:100AF0008D18A01BAC420AD0054B21781868054B15
:100B000001341B6898470028F3DA0120404270BD89
:100B1000380200203402002070B594B008AC2000E8
:100B2000284B9847042180222173C0210023264DA1
:100B3000520062804901FF3AA36023716270E18133
:100B40002275A3742200214B2149280098472B6865
:100B50005A7E52B2002AFBDB0F229A751A76197858
:100B60000D3A0A431A702A68537E5BB2002BFBDBF6
:100B70006846184B98476A4627230024164E694654
:100B800053703000154B94709847012302A90B70E5
:100B90004B71CB700F330B812B684C701A33CB60C9
:100BA0000F4B8C708C71CC710C710E4C20330B611F
:100BB00020000D4B4C619847210030000B4B9847AB
:100BC00014B070BD5501000008010020990100001B
:100BD000004000421D050000100100202D0500000E
:100BE0002C01002040020020E50600008D070000D7
:100BF00010B5094B1B685A7E52B2002AFBDB022259
:100C0000197B0A431A735A7E52B2002AFBDB03484F
:100C1000034B984710BDC04608010020100100207A
:100C2000590600000023180004495A5A023380185C
:100C3000202BFAD1000980B27047C0462C01002059
:100C400010B5044B9847044B98470449044B984708
:100C500010BDC046250C0000F129000009F90C3A2E
:100C60009923000073B56B469C1D002306000D0000
:100C7000238021003000034B98470028F9D12388B6
:100C80002B7073BD7310000070B504000D00A9B285
:100C90002000024B98470028F9D170BD5110000088
:100CA000F8B580232D4ADB051360FF2301250024BE
:100CB0001381531DDD77931DDD77D31DDC77130082
:100CC0000833DC7713002C331C7013002D331C7099
:100CD00013239376224B234E1363234B54605363A9
:100CE00001235B429363D36380235B03D360E123DF
:100CF0005B0213621D4B9472D4729462546114822D
:100D0000D476147614775476547719491E60194BAB
:100D1000300019601849194B19601949194B984747
:100D2000194F21003B689868184B98473B68210091
:100D30005868164B98473468154B200098471F2376
:100D400018408540134B1D603268D369002BFCD1DD
:100D50002268023313432360F8BDC0464C010020D3
:100D60000200160050020020020017003802002086
:100D7000890C000034020020650C000030020020C5
:100D800000140042990D00001800002041490000A5
:100D90008112000000E100E0F0B5070093B09E4B27
:100DA000396008001400049198470122049B060052
:100DB0001B680520134200D00AE1049B17301D6810
:100DC00002231D4000D003E1F3181B3898400300B4
:100DD000924A1436116AF6B20B43136223002D3384
:100DE00002931B780CA90B7030008D4B9847300094
:100DF0008C4B9847029B290018788B4B9847E37AD5
:100E000008267B71631DDB7FBB71A31DDB7FFB713C
:100E1000E37E3B72237F7B723B68039318007E4B1B
:100E200098470EAB1D80238A143002938023029AC8
:100E3000DB019A4214D008D8802310269B019A42E5
:100E400000D1C8E0102600250AE0C023029ADB0189
:100E50009A4200D1BEE0802303261B029A42F1D1C0
:100E600023680693E368079363690893237E0993D5
:100E7000E31DDB7F0A93636805932300059A08331B
:100E8000002A00D1A9E080220599520591420ED195
:100E9000DB7F002B0BD1654BC0B2256A98470EAAA9
:100EA0000100634B28009847002800D090E0637E43
:100EB000002B02D0A37E039A93730EAE3388039A5D
:100EC0009381079A069B1343089A1343059A134389
:100ED000029A1343099A120213430A9A52071343C0
:100EE00022000832D27F002A01D104321343627EED
:100EF000217F920249020A43617FE07A09020A4394
:100F0000611DC97F49040A43A11DC97F09040A4321
:100F1000A17A01430A432189FF2900D173E080208F
:100F2000400403430A4321002C310978002903D1EE
:100F300040498978890701D580210B433868C16908
:100F40000029FCD103994A603968CA69002AFCD19A
:100F500003990DAD0B6080232B70236B6A700E9389
:100F6000636BEA707360A36BAA70B360E36B1400E9
:100F7000F360A300F058E1B2002802D104982E4B90
:100F80009847431C05D02870000CC0B229002B4B99
:100F900098470134042CECD13B0000243033FC850D
:100FA000FC603C617C61BC61FC613C62BC627C6257
:100FB000BC859C701C705C70DC703868164B984760
:100FC00005001F4B1F49984720001F4BAD00EF50F5
:100FD00013B0F0BD0826012542E7DB7F002B07D0C8
:100FE0002B000096A16A206A0EAA184DA8475BE75D
:100FF000236AC0B20B930D4B9847009601002B005B
:101000000EAA0B98F1E7E17E002900D18BE7802141
:10101000C9040B4387E7C0467D0A00000004004076
:101020004D180000C5170000DD0800006918000019
:101030001D080000002000412109000021190000C6
:1010400049120000DD100000840200204508000065
:10105000C2791C23002A0AD0C28D173B002A06D170
:10106000036802321985197E1142FCD00023180052
:10107000704710B582791C23002A11D0828D173B4E
:10108000002A0DD102680420147E044208D0538B3C
:10109000DBB29C061DD00224234203D01A235483C2
:1010A000180010BD034202D050831E23F8E7012030
:1010B000034202D050831323F2E71020034202D0F0
:1010C00050834223ECE72020034202D05083412387
:1010D000E6E7138D0B800023E2E70000F8B5584BDC
:1010E0008000C4582568EB69002BFCD12B7EAF7DB6
:1010F0001F40230030331A785E78012316401F42C8
:1011000019D0E28D002A00D172E0A26A511C137836
:10111000A1626179DBB2012964D09BB2DB05DB0DF2
:101120002B85E38D013B9BB2E385002B03D101337B
:101130002B750133AB7502231F4209D02B75230099
:10114000002233331A70F30702D52000E368984772
:1011500004231F4227D0A28D002A00D16DE06B8BA3
:10116000DBB21A0746D43F22134045D002221A218F
:1011700013420FD104221E2113420BD1012213214D
:10118000134207D110224221134203D120221342DD
:1011900004D041212300323319706A83730702D5CA
:1011A00020006369984710231F4206D02B752B76C9
:1011B0001E4202D02000E369984720231F4206D038
:1011C0002B752B76330702D52000A3699847082397
:1011D0001F4206D02B752B76B30602D5236A20005A
:1011E0009847F8BD5178023209020B43A26295E795
:1011F0002B75A0E73722B7E72B8D616ADB05DB0D86
:10120000DAB20A70626A511C61626179012904D103
:101210001B0A5370636A01336362A38D013B9BB267
:10122000A385002BBFD104222A752200323213700D
:10123000B307B8D520002369B4E72B75B3E7C046E0
:101240008402002070470000F0B5094C094A237859
:10125000002B09D11E00084F084DD750EE50043323
:10126000182BFAD1173B237080001150F0BDC046F7
:101270008C01002090010020451200008402002013
:1012800007B509236A461370013353700133937015
:101290000133D3700133137101335371024B9847FB
:1012A0006B4618560EBDC0467D0A000010B5024BB5
:1012B00000201B68984710BD9001002010B5024B1C
:1012C00001205B68984710BD9001002010B5024BCB
:1012D00002209B68984710BD9001002010B5024B7A
:1012E0000320DB68984710BD9001002010B5024B29
:1012F00004201B69984710BD9001002010B5024BD7
:1013000005205B69984710BD9001002070B5094B1E
:1013100000209847FA21084C89000500A047074B98
:10132000074918602800A0470522064B1860064BA5
:101330001A6070BD3D1700005D2100000C00002008
:1013400040420F001000002010E000E030B5802483
:101350000021074B64021A68064B013800D230BDE9
:10136000002AFAD05A6099601D682542FCD0F4E743
:101370000C00002010E000E0094B196800290BD197
:10138000EFF31080074A002805D172B6BFF35F8FD4
:1013900005490870012111701A6801321A607047FE
:1013A000A8010020AC01002014000020084B1A689E
:1013B000013A1A601B68002B09D1064B1B78002BE1
:1013C00005D00122044B1A70BFF35F8F62B67047DD
:1013D000A8010020AC01002014000020F7B5012571
:1013E000002701AC084E21003E206570A7702570D3
:1013F000B0478022054BD2051A6021000F202770CC
:101400006570B047F7BDC046111400009844004114
:1014100007B5802201AB1A700A785A704A789A7020
:101420008A781900DA70014B984707BD211900002E
:1014300010230249CA681A42FCD0704700080040D5
:1014400070B5082806D800F07FFE08050530301278
:101450000B1528000024200070BD164B1C69FAE70C
:10146000154B164C1B6A9B059B0FDC40F3E7114B99
:101470005C69F0E70F4D00242B689B07EBD5104B00
:10148000984724222B681340042B11D120000D4BC8
:101490009847AC68A4B24443DDE70B4B00241B78AB
:1014A0005B07D8D5034BDC68D5E780242402D2E75C
:1014B000064CD0E7B00100200008004000127A007E
:1014C000311400006918000050080040006CDC0274
:1014D00070B5847802784578012040260540204088
:1014E00080240849AD010B6AC001B3432B43A343D9
:1014F00003430320024004481202034013430B62DB
:1015000070BDC04600080040FFFCFFFFF8B508288A
:1015100006D800F019FE1405050C0E1A0720340039
:101520001720F8BD0223194A116A0B4313620020E9
:10153000F7E70223154A91690B439361F7E702230A
:10154000124A118A0B431382F1E702230F4A918A50
:101550000B439382EBE7022200240D4E0B4D3368C0
:101560000C4F13433360AA84B847B368EB627368C7
:10157000AB62AC84B84733689BB2AB84D7E7022335
:10158000054A11780B431370D1E7C04600080040AC
:10159000B001002031140000440800407FB5C22291
:1015A0001E21194BD2009A60184A0024536801ADDD
:1015B0008B43536001232B70E0B22900144B01349C
:1015C0009847252CF8D100246B4601265C709E704C
:1015D0001C7068460F4B98470F4B062098470F4BDF
:1015E00098470F4B29001C725C729C72DC720623B8
:1015F00020002B700B4B6E606C702C726C729847D5
:101600002000094B98477FBD000800400040004182
:101610004D180000D11400000D150000391600000F
:101620000004004059160000FD160000014B5878D8
:10163000C0097047000C00400823054A91690B431C
:1016400093610123034A137011781942FCD170474A
:1016500000040040000C0040F8B50C784B782402E0
:10166000060005000443002B02D08023DB021C434C
:101670004B7A002B02D080231B031C434B68012BA9
:1016800012D95D1E1D400222002D06D01D028023AE
:1016900035439B0207E0013552009A42FBD3802379
:1016A0002D0235435B031C430B7A002B02D08023B1
:1016B0009B031C430C4FB8470028FBD10B4B9847AA
:1016C0000B4B1E70B8470028FCD10A4B9D601D00D3
:1016D000B8470028FCD180226B68520213401C439B
:1016E0006C60054B9847F8BD2D160000791300007B
:1016F000080C0040000C0040AD13000070B5050060
:10170000094CA0470028FBD1084B9847084B1D7097
:10171000A0470028FCD18023064A5B0251680B4396
:101720005360054B984770BD2D16000079130000DB
:10173000040C0040000C0040AD130000F7B507009A
:10174000184EB0470028FBD1174B9847174B1F7016
:101750000193B0470028FCD1154D164B6868C004B2
:10176000C00E98470400019B1F706B68DB02DB0F03
:101770000193114B1F70B0470028FCD1AD680F4B8F
:101780009847019B2D022D0C002B08D1012D04D967
:10179000200029000A4B984704002000FEBD0135B7
:1017A000EC40FAE72D16000079130000040C00400D
:1017B000000C004041140000080C0040AD13000074
:1017C0005D21000010B50400064B9847064B074A00
:1017D0001C7080235188DB010B435380044B9847D6
:1017E00010BDC04679130000020C0040000C004000
:1017F000AD13000010B504000E4B98470E4B0F4A76
:101800001C700F4B0F4C58885988000511405980A7
:101810005988000F2140598011008022D2015C8834
:101820001442FCD15A8800020A4002435A80064BF7
:10183000984710BD79130000020C0040FFF0FFFF35
:10184000000C0040FFBFFFFFAD13000010B50C7887
:10185000034B240204439847024BA4B25C8010BDA2
:10186000F5170000000C004010B50400064B984727
:10187000064B1C70064B5C88064B2405240F9847CA
:101880002000054B984710BD79130000020C004062
:10189000000C0040AD1300003D170000D37830B5B8
:1018A000002B35D11478802C03D0802324065B02D2
:1018B000234302255478AC4306D19478002C24D1DC
:1018C0008024A402234341605478013C012C01D8B8
:1018D000124C2340A0248DB2E4052C431C438462A7
:1018E000D0240D0C24062C431C438462D478002C95
:1018F0000AD15B0303D59378012B0CD18161537816
:10190000013B012B00D8816030BDC024E402D9E73F
:1019100041600023DEE74161F1E7C046FFFFFBFFC6
:1019200010B503000A004409C1090020814202D118
:101930000449E00140181F210B401E399940024B19
:10194000984710BD004400419D18000070470000FA
:1019500010B5054B9847054B9847054B9847054BE5
:101960009847054B984710BD9D150000DD130000FA
:101970004D1900004D1900004D190000FEE7000050
:101980002148224970B5884204D00023204CCA184F
:10199000A24232D300211F4B1F4A934231D3FF2171
:1019A0001E4B1F4A8B43936002220C2508243026CD
:1019B0001C4B1D485A62C378FC398B431343C370D8
:1019C000C378AB432343C370184B987BB0430600E6
:1019D000202030439873987BA84304439C73987BE2
:1019E000884302439A738023114A51680B43536022
:1019F000104B9847104B9847FEE7C55804331560C5
:101A0000C5E702C3C9E7C046545B000000000020E0
:101A10007C00002080000020A002002000000000C8
:101A200000ED00E0FC700041005000410048004122
:101A300000400041CD470000751A0000054B020030
:101A40001968002901D104491960186882181A60C0
:101A50007047C046C8010020A0220020012040425B
:101A6000704780239B0100204B6070470120704726
:101A700000207047F7B5414B9847414B98470122EA
:101A8000404B1A70BFF35F8F62B63F4B98473F4B96
:101A900098473F4B98471B213E4C3F48A0471B218E
:101AA0003E48A0473E483F4B98473F4B98473F4BE7
:101AB0003F49061C98473F4FB84700900191301CA2
:101AC000B8473D4C02000B003C483D49A0473D4C07
:101AD00002000B0000980199A0473B4B98473B4BF5
:101AE00098473B4C3B4A3C4BA0473C4B98473C4AB1
:101AF0003C4BA0473C4C3D4A3D4BA047314C02007B
:101B00000B0000203B49A0473B4CA047B8472B4A5D
:101B10003A4B294DA847A047394D071C301CA84710
:101B2000384B04009847384B011C301C98471F4B1A
:101B300036499847A84721000200164C3448A04770
:101B4000381CA8472F4B060098472F4B011C381C08
:101B50009847A847FA229200424331002D48A047F7
:101B6000FA202D4B400098471B212C48A0471B21F1
:101B70000A48A0471B212A48A04796E751190000B0
:101B80000D13000014000020A10C0000190B000030
:101B9000F10B000039480000585900005E59000060
:101BA000635900002D490000410C000099230000FA
:101BB00000401C46CD450000053E00006666666696
:101BC00066660A409D3000005D2300005D45000010
:101BD000053900002D431CEBE2361A3F251C00009E
:101BE000D81C26619F32313F7D2A00005DE5F7A0B9
:101BF000E1796B3F0000F03F7146000066127140D2
:101C00001129000051290000D925000000007A4464
:101C10009F590000B15900004D130000C659000043
:101C2000CC590000F0B5C64600B58CB004000D00DC
:101C300000F080F83A4B06001B780F005BB2984624
:101C400001330FD022002B002000290002F0F0FB0E
:101C5000002807D1002200232000290000F040FBCB
:101C6000002805D0300039000CB004BC9046F0BD0F
:101C70002C4B0A90039343460494059506940795CC
:101C8000002B1AD1E022284B12060892099320005B
:101C900000220023290000F009FB002838D002238D
:101CA000029302A800F048FA002817D00A9B01937B
:101CB000002B18D1089E099FD4E700221B4B20005F
:101CC0000892099329000022002300F0EFFA00286F
:101CD0000FD0022302934346022BE2D102F070FDA3
:101CE00022230360E2E702F06BFD0A9B019303608D
:101CF000E0E7012302934346022B0BD102F060FD83
:101D0000212303600A4800F019FA08900991CDE7F1
:101D10000123029302A800F00FFA0028F2D1EDE7A8
:101D200015000020D4590000FFFFEFC70000F0FFAE
:101D3000D8590000F0B5D6464F464646C0B5DA4AF7
:101D400088B00B00914255DC4A005208024300D192
:101D5000EFE0002900DA79E1D44B002201F0D2FD56
:101D60003625D34C0B006D42A34247DC1A15D14CEB
:101D70001B031B0B9846A4468024CF4B64034344AB
:101D80002340CE4C624452195C4045461B1599468F
:101D90002543CA4B29009144002202F033F8434600
:101DA00002331B0306000F001B0B0022022B2FDC4B
:101DB000002300F07BFA002800D1C1E04B46002B45
:101DC00000D14CE1484602F087FBBD4ABD4B040000
:101DD0000D0001F097FDBC4A06000F00BB4B200030
:101DE000290001F08FFD02000B003000390000F0E7
:101DF00045FE07E0AE4C0025A342B7DD02000B0014
:101E000000F03CFE08B01CBC90469946A246F0BDCE
:101E10008023DB0500F032FE02000B0030003900A9
:101E200001F03CF9040048460D0002F055FB220089
:101E3000029003912B00200029000494059501F0E5
:101E400061FD04000D00A24B020043449A460B00C2
:101E50000094019501F056FD04000D009D4A9E4B33
:101E600001F050FD9D4A9E4B00F008FE22002B0021
:101E700001F048FD9B4A9C4B00F000FE22002B0025
:101E800001F040FD994A9A4B00F0F8FD009A019B41
:101E900001F038FD974A00900191974B20002900EE
:101EA00001F030FD954A964B00F0E8FD22002B0032
:101EB00001F028FD934A944B00F0E0FD22002B0036
:101EC00001F020FD0B0002000098019900F0D6FD02
:101ED0000D0041468D4B04005B1A51460B43002B0D
:101EE00054DD00228A4B3000390001F00BFD320036
:101EF0003B0001F007FD4B460A00010000910192F2
:101F0000002B72D1130029000200200000F0B6FD62
:101F1000049A059B01F0F6FC02000B000098019961
:101F200001F070FF02000B003000390001F06AFF81
:101F300068E7002200230020764901F0AFF861E74E
:101F4000754A764B3000390001F0DCFC02000B00D2
:101F500000206F4901F056FF320004000D003B00E5
:101F60003000390001F0CEFC0B00020029002000F7
:101F700001F0C8FC4B4604000D00002B72D102009A
:101F80000B003000390001F03DFF3BE74B46002BD2
:101F900000D1C5E002980399494A4A4B01F0B2FCCE
:101FA0002200009001912B003000390001F02AFF3F
:101FB000049A059B01F0A6FC434A04000D00029818
:101FC0000399424B01F09EFC02000B002000290007
:101FD00001F018FF32003B0001F014FF02000B007B
:101FE0000098019901F00EFF0CE7354A354B029835
:101FF000039901F087FC009A019B0690079120004D
:10200000290000F03BFD049A059B01F07BFC2E4A61
:1020100004000D00029803992C4B01F073FC0200A0
:102020000B002000290000F029FD02000B000098A1
:10203000019901F0E7FE32003B0001F0E3FE0200EF
:102040000B000698079901F0DDFEDBE602000B00AD
:1020500001F0D8FE0022002301F020F8D2E6002093
:102060000021CFE6484602F037FA154A154B00909A
:10207000019101F047FC144A0290039100980199E4
:10208000124B01F03FFC02000B002000290001F080
:10209000B9FE32003B0001F0B5FE02000B000298D1
:1020A000039901F0AFFEADE6FFFF0F0000005043C3
:1020B000FFFFEF7F01FCFFFF645F09000000F03FBE
:1020C0000000E0FE422EE63F763C7935EF39EA3DEE
:1020D00086EBF9FF44523EDF12F1C23FDE03CB969E
:1020E0006446C73F599322942449D23F935555558E
:1020F0005555E53F9FC678D0099AC33FAF788E1DEE
:10210000C571CC3F04FA97999999D93F51B8060007
:102110000000E03F000050C3555555555555D53F7B
:1021200022002B003000390001F06CFE049A059B60
:1021300001F0E8FBF6E6C0460020704700200149A8
:102140007047C0460000F87F02B471464908490054
:10215000095C49008E4402BC7047C0460022430817
:102160008B4274D303098B425FD3030A8B4244D35F
:10217000030B8B4228D3030C8B420DD3FF220902A1
:1021800012BA030C8B4202D31212090265D0030B60
:102190008B4219D300E0090AC30B8B4201D3CB0356
:1021A000C01A5241830B8B4201D38B03C01A524198
:1021B000430B8B4201D34B03C01A5241030B8B429A
:1021C00001D30B03C01A5241C30A8B4201D3CB0285
:1021D000C01A5241830A8B4201D38B02C01A52416A
:1021E000430A8B4201D34B02C01A5241030A8B426D
:1021F00001D30B02C01A5241CDD2C3098B4201D385
:10220000CB01C01A524183098B4201D38B01C01A02
:10221000524143098B4201D34B01C01A5241030979
:102220008B4201D30B01C01A5241C3088B4201D328
:10223000CB00C01A524183088B4201D38B00C01AD5
:10224000524143088B4201D34B00C01A5241411AFC
:1022500000D20146524110467047FFE701B5002009
:1022600000F006F802BDC0460029F7D076E77047B7
:102270007047C0469140031C90409C46203A9340D2
:10228000194352426346D340194370478446101C99
:1022900062468C46191C634600E0C0461FB501F03B
:1022A000CFFA002801D40021C8421FBD10B501F0AB
:1022B00029FA4042013010BD10B501F0C1FA0028E2
:1022C00001DB002010BD012010BDC04610B501F09B
:1022D000B7FA002801DD002010BD012010BDC04666
:1022E00010B501F049FA002801DC002010BD0120E2
:1022F00010BDC04610B501F03FFA002801DA0020F9
:1023000010BD012010BDC046F0B5CE4647461504AD
:102310002D0C2E0080B50704140C3F0C9946030CBD
:102320007E435D43674363437F19340CE4199C4645
:10233000A54203D980235B029846C4444B465143CF
:1023400043433604360C250C24046544A41959185B
:10235000491920000CBC90469946F0BD70B500228A
:102360000C4B04000D00FFF7C5FF002804D120002E
:10237000290002F07DF870BD064B002220002900E4
:1023800001F040FD02F074F880231B069C46604477
:10239000F1E7C0460000E041F8B557464E464546D5
:1023A000DE46E0B54702460088467F0A360EC40F77
:1023B000002E47D0FF2E24D0FB008027FF041F43B0
:1023C000002399469A467F3E43465D025800DB0F44
:1023D0006D0A000E984643D0FF283BD0EB008025C5
:1023E0000022ED041D437F383618731C41469B467E
:1023F0004B46614013430F2B64D875489B00C3586C
:102400009F46002F42D108239946063BFF269A4655
:10241000DAE74146022A28D0032A00D1CEE0012A79
:1024200000D0ACE0114000200022CCB24002D20526
:10243000400AE407104320433CBC90469946A2461C
:10244000AB46F8BD002F15D104239946033B002667
:102450009A46B9E7FF200222002DC5D00322C3E728
:10246000002D19D100200122BEE70124FF220C40DB
:102470000020DBE7380002F085F97626431F9F40F5
:1024800000237642361A99469A469DE70C239946D0
:10249000093BFF269A4697E7280002F073F9431F8D
:1024A0009D4076235B42181A00229DE7802000247D
:1024B000C003FF22BAE73D005246ABE73D002100D2
:1024C0005246A7E73B0C9C462A04120C2B0C140026
:1024D000604665463F043F0C7C4342435D437B437B
:1024E000270C9B18FF18BA4203D980235B029C4635
:1024F000654424043A04240C121993015C1EA34180
:102500003F0C920E7D191A43AD0115432B0104D5E2
:1025100001235E466A081D40154332007F32002ABF
:1025200025DD6B0704D00F232B40042B00D004358E
:102530002B0103D53200274B80321D40FE2A94DC4C
:102540000124A801400AD2B20C406FE78020C003EA
:10255000074207D0054205D128434002400A4446BD
:10256000FF2263E738434002400AFF225EE701246E
:10257000A31A1B2B05DD0C400022002056E75E4607
:10258000CBE72A002020DA40C31A9D402B005D1EB5
:10259000AB4113435A0704D00F221A40042A00D03B
:1025A00004335A0104D5012401220C4000203DE7E8
:1025B00001249B01580A0C40002237E780200124A7
:1025C000C00328434002400A0C40FF222EE7C046C9
:1025D000DC590000FFFFFFF7F0B54F46D6464646F0
:1025E0004400C0B5C20F47024802400A844666460E
:1025F0007B0A4800C90F9A46240E1500DB00000E26
:102600008946F600FF2800D18FE001214F464F4058
:102610003900914266D0221A002A00DC9DE0002891
:102620003DD1002E00D18BE0511E002900D0B5E035
:1026300001249B1B5A0144D59B019F09380002F0DD
:10264000A1F805388740844200DD96E0041B3A007B
:1026500020200134E240041BA7403B005F1EBB4129
:10266000002413435A0704D00F221A40042A00D032
:1026700004335A0127D50134FF2C00D179E001221F
:102680009B015B0AE4B22A405B02E405580AD207C8
:10269000204310431CBC90469946A246F0BDFF2C37
:1026A000E0D08021C9040E431B2A7BDC31002020AE
:1026B000D140821A9640721E96410E439B1B5A01CE
:1026C000BAD45A07D0D10122DF082A40FF2C33D1D7
:1026D000002F00D1A8E08023DB033B435B025B0AB1
:1026E000FF24D1E7211A00294CDD00282AD0FF2C35
:1026F000B8D08020C00406431B2900DDAFE03000C5
:102700002027C840791A8E40711E8E4106439B19BE
:102710005901D6D50134FF2C00D185E001227A4938
:102720001A405B080B4013439CE7002E00D070E773
:102730006BE73B1EC5D100227B025B0AE4B2A3E734
:1027400014008FE7002E4DD0481E002857D19B194A
:1027500001245A01B5D50224E0E7002A25D1621CE4
:10276000D2B2012A72DD9F1B7A0135D5F71A0D000E
:1027700064E7012200232A4086E73B00634A241ACB
:1027800013406FE700296CD1611CC8B201284EDDEF
:10279000FF2949D09B195B080C0063E7FF2A41D051
:1027A0000A0081E701269B1B89E7002C1CD0FF282B
:1027B00021D08024E404524223431B2A00DD96E00A
:1027C0001C002025D440AA1A93405A1E934123434B
:1027D000F31A04000D002DE7002F00D02EE7002291
:1027E0000024A9E70C003DE7002B58D0D243002A73
:1027F000EED0FF28E1D13300FF240D0032E7FF299E
:1028000010D0010078E7002B6ED0FF24002E00D1FD
:1028100028E780225146D203114203D0614611427B
:1028200000D13300FF241DE7FF2400232CE7002CF8
:10283000E9D1002B63D0002E00D113E79B195A0178
:1028400000D43EE7314A0C0013400BE7002C1ED1A8
:10285000002B2FD1002E4FD033000D0002E70126B0
:1028600055E7002C1FD1002B43D0C94300290BD0C2
:10287000FF2839D01B2944DC1C002027CC40791AC2
:102880008B40591E8B4123439B19040040E7002BCA
:102890001AD1002E24D180270022FF031BE733002A
:1028A00004000D00DEE6FF281ED08024E404494227
:1028B0002343DFE7002E00D1D4E69F1B7A0100D42A
:1028C00037E7F31A0D00CDE6FF24002E00D1C9E64C
:1028D00080225046D2031042A4D060461042A1D1BB
:1028E00033000D00FF24BDE63300FF24BAE60123C8
:1028F0006EE733000400B5E6002700221CE7330032
:10290000B0E60123C0E7C046FFFFFF7DFFFFFFFBEE
:1029100041024300C20F490A1B0E00207E2B0DDD31
:102920009D2B0CDC802000040143952B0ADC9620B3
:10293000C31AD9404842002A00D108007047034B0F
:10294000D018FBE7963B9940F4E7C046FFFFFF7FB6
:1029500070B5002830D0C317C4185C40C50F2000E4
:1029600001F010FF9E231B1A962B0DDC9622D21A23
:1029700094402A006402640ADBB26402DB05600A48
:10298000D2071843104370BD992B19DC9922D21A33
:10299000002A29DD94402200144C1440510704D031
:1029A0000F210A40042A00D00434620113D4A40188
:1029B000640ADBB22A00E0E7002200230024DCE7FF
:1029C00005222100121AD140B922D21A9440621E67
:1029D00094410C43DAE7054B2A001C409F23A401D5
:1029E0001B1A640ADBB2C8E72200D5E7FFFFFFFB32
:1029F00010B5041E27D001F0C5FE9E231B1A962B8E
:102A00000ADC9622D21A94406402640ADBB26402A1
:102A1000DB05600A184310BD992B17DC9922D21AE6
:102A2000002A27DD94402200134C1440510704D0A3
:102A30000F210A40042A00D00434620112D4A401F8
:102A4000640ADBB2E3E700230024E0E7B9222100B7
:102A5000D21A91400A00511E8A410521091ACC4020
:102A60001443DBE7044B1C409F23A4011B1A640A98
:102A7000DBB2CCE72200D7E7FFFFFFFBF8B5454606
:102A8000DE4657464E460C03E0B54E00C90F884659
:102A90000D00610A440F0C43C70019035800DB0FF7
:102AA0009B464B0A510F0B43760D400D1900D20087
:102AB000D84500D1AEE0351A002D00DCF6E0002844
:102AC0000FD1134300D1DBE06B1E002B00D037E1A8
:102AD000BA1A9742BF41641A7F42E41B01261700CD
:102AE00024E0C64B9E424DD080231B041943382D51
:102AF00000DD07E11F2D00DD38E12020431B9A4651
:102B00000B0050468340994613004846EB4018435B
:102B1000030050468240501E8241E9401A43BA1ACF
:102B2000611A9742A441170064420C1B230262D52C
:102B30006402650A002D00D1DFE0280001F022FECA
:102B40000300083B1F2B00DDD2E020223C00D21AFC
:102B50009D40D4409F4025439E4200DDC4E09E1B23
:102B6000731C1F2B00DDF1E0202238002900D21A4F
:102B7000D840914097402C000143781E8741DC40AB
:102B800000260F437B0709D00F233B40042B05D0C1
:102B90003B1DBB42BF417F42E4191F0023022CD5DD
:102BA000964B01369E4200D19AE04546944BFF0871
:102BB0001C406007760564020743240B760D002154
:102BC0002403230B0C0D8F4A24051C4314403305AA
:102BD00023435B00ED075B082B43380019003CBC26
:102BE00090469946A246AB46F8BD6446044300D1E0
:102BF00011E2040067467B07C6D145466007FF081F
:102C00000743E4087D4B9E4230D024037605240B15
:102C1000760DD4E7331A9A46002B78DD002831D0A0
:102C200076488642AED08020000401435346382BBC
:102C300000DCE9E00A43511E8A410021D219BA4260
:102C4000BF4109197C4217000C192302D3D56B4BE5
:102C500001369E4200D13AE10120694B1C407B08BD
:102C600007401F43E007074364088BE723003B430B
:102C700000D1CBE18022120314432403240B9EE7EE
:102C80002E007FE70800104300D1B4E0581E002852
:102C900000D0DEE0BA18BA429B4164185B42E418E7
:102CA000170001262302A6D50226D5E7002D6ED1F6
:102CB000701C4005400D012800DCF9E0B81A84467C
:102CC00087428041E51A40422D1A280200D489E04B
:102CD000D71BBA4292411C1B5242A51AD84629E77B
:102CE0004546002400276AE7454CF61A2C4049E780
:102CF0003D002838854000272EE7380001F042FDCE
:102D000020301DE70A43511E8A41002107E7002BAE
:102D100000D0F3E0701C43055B0D012B00DCADE03F
:102D2000364B984200D1D1E0BA18BA42BF4164187C
:102D30007F42E419E707520817436408060021E7B9
:102D40002E48854200D193E01D00D0E629001F3EA9
:102D5000F140202B00D18DE04022D31A9D402F431B
:102D60007D1EAF4100240F43002644E72B000800DE
:102D7000203BD8400300202D00D17DE04020451BA2
:102D8000A9400A43511E8A4100211A43C7E6002E7A
:102D900050D01A4EB04257D080266B429946360426
:102DA00034434B46382B00DDD6E01F2B00DD35E1E8
:102DB0002026F51A2600AE40B2463E00DE40AC4664
:102DC000350056462E436546AF407D1EAF41DC4080
:102DD0003743D71BBA4292410C1B5242A41A060039
:102DE000D846A3E6644667462C4300D0A2E60025F9
:102DF0000026002706E71E00C4E6C046FF070000C5
:102E0000FFFF7FFFFFFF0F801F2B63DC2020C31A13
:102E1000080098409C46834653461000D840030063
:102E20005846184363469A40531E9A4153460243FC
:102E3000D94003E726003E4306D0EB439946002BDA
:102E4000C7D0944EB042ACD10C0017000600D84653
:102E500098E6904B9A450BD08246E7E6002800D0D2
:102E60009EE01800104300D1E9E01C001700D8468E
:102E7000884E87E6002572E7002182E723003B4366
:102E8000002E00D0ABE0002B00D1E7E00B00134395
:102E900000D177E6BA18BA42BF4164187F42E419FC
:102EA000230200D4F2E07C4B17001C40060069E6C8
:102EB00020003843002ED1D100285BD11C001443E0
:102EC00000D1A8E01C001700D8465BE606000024ED
:102ED000002797E650460B002038C34099465346DA
:102EE000202B00D195E0402350461B1A99400A43FD
:102EF000511E8A414B4600211A439FE6002E30D1D5
:102F000026003E4367D0DB439A46002B1CD0614E1F
:102F1000B04260D05346382B00DD96E01F2B00DD19
:102F20009FE02026F31A26009E409C46B346534657
:102F30003E00DE4033005E461E4363469F407B1EDC
:102F40009F415346DC403743BF1897429241641873
:102F50005242A418060078E627437C1EA7410024AD
:102F600037E74C4EB04236D080265B4236049A4654
:102F70003443CFE71800104300D103E6B81A844663
:102F80006745AD41E01A6D42401B050200D42CE6B6
:102F9000D71BBA4292411C1B5242A41AD846F1E5F3
:102FA0001800104300D163E7F80867070743802043
:102FB000E4080003044208D0DD08054205D1D20828
:102FC000590711430F002C00D8467B0FE4001C4327
:102FD000FF00304ED6E50C0017000600D2E5002BAE
:102FE00038D00B00134300D142E7F80867070743C6
:102FF0008020E40800030442E7D0CB080342E4D178
:10300000D208490711430F001C00DEE70027002407
:10301000D5E500216BE700250027F3E54E462500A6
:10302000203EF5404B462E00202B2DD04025ED1A9A
:10303000AC4027437C1EA74100243743C9E68024C7
:1030400000252403134E0027DCE527437C1EA741FF
:10305000002479E70C0017000E4E93E50C001700D2
:1030600090E556462300203EF34099465346202BD8
:103070000ED0402356469B1B9C4027437C1EA741F5
:103080004B4600241F435FE70024D2E71700B2E558
:103090000024F2E7FF070000FFFF7FFFF0B557466F
:1030A0004546DE464E46E0B54C000E0387B08346EB
:1030B00092461D008046360B640DCF0F002C4FD07A
:1030C0006F4B9C4235D08023420F1B04F600134304
:1030D00033439946C30098466A4B00269C4600231A
:1030E000644403932B031B0B9B466B00ED0F504670
:1030F0005B0D01955ED0624A934253D05A46D1008F
:103100008022400F120402430A4393465246D100E4
:103110005C4A94460022634438006840844602902A
:10312000E41A16430F2E00D9B4E0574BB6009B5952
:103130009F460300334399466CD1002398460233DF
:1031400008260393CEE7CB464146039A0197022A0D
:1031500065D1019B4A4C9C460023002298466BE0B7
:103160000300334399464ED0002E00D1BCE130001D
:1031700001F008FB03000B3B1C2B00DDACE11D2222
:10318000D31A5A460100DA4008398E4013003343FF
:1031900099465B468B40984600233C4C0026241AF7
:1031A00003939FE751465A46114329D10022934683
:1031B0000232B1E7594601431ED05B46002B00D1D5
:1031C0009EE1584601F0DEFA03000B3B1C2B00DDAC
:1031D0008FE102005946083A91408B461D21CB1AD7
:1031E0005146D9400B0059460B4351469B469140EE
:1031F000264B00221B1A8FE7002301229B468BE7F8
:103200005146032288E70023984601330426002410
:10321000039367E70323B14603930C2662E7032A6F
:1032200000D15CE2019B012A00D0E4E113409C46FE
:10323000002300240022984600211203130B0A0DDC
:1032400012051A432305124C40462240134362469E
:103250005B00D2075B081343190007B03CBC9046E3
:103260009946A246AB46F0BD002380229C4612033D
:103270009846034CE0E70023014C00229846DBE728
:10328000FF07000001FCFFFF1C5A00000DFCFFFFC0
:10329000FFFF0F80D94500D939E100D134E1002387
:1032A00046464D469A46013C5B460A0E1B021A43AF
:1032B0000B02170C039313041B0C390028009046D3
:1032C0000193FEF74BFF0200019B83465A432800FF
:1032D00039009146FEF7C8FF350C09040D43A94596
:1032E0000DD95B464544013BA84500D93AE1A945C3
:1032F00000D837E102235B429C464544E3444B46F9
:10330000EB1A390018000493FEF728FF019B050013
:103310004343390004989946FEF7A6FF3304090495
:103320001B0C0B43994509D943446A1E984500D9A3
:103330001AE1994500D817E1023D43444A469B1AD9
:103340005A4612042A4303999346100C0A0C9146DC
:1033500009045A46090C4E460D001204120C45434E
:10336000059151437243704352190E0CB2189542A5
:1033700003D980256D02AC466044150C0904120483
:10338000090C28185218834200D2CEE000D1C8E0C0
:103390001D1A53469E1AB24592415242AB1A9A46A2
:1033A000984500D117E139001800FEF7D7FE019BC0
:1033B00005004343390050460493FEF755FF049837
:1033C0000B04310C1943884209D941446B1E8845CE
:1033D00000D907E1884200D804E1023D4144049B42
:1033E000CB1A180039000493FEF7B8FE019B824601
:1033F0004343390004980193FEF736FF01980B040C
:103400003104090C194388420DD953464144013B0C
:10341000884500D9E8E0884200D8E5E002235B4215
:103420009C464144E244019B2D04CE1A5146294357
:10343000059D4F462A000B04080C1B0C5A434543BC
:103440007B4378435B19170CFB189D4203D98025F9
:103450006D02AC4660441D0C12041B04120C2818AB
:103460009B18864200D293E000D18EE001231943DD
:10347000A04BE318002B00DC99E04A0700D09EE047
:103480005A46D20106D55A469B4B1A408023934692
:10349000DB00E318994A934268DD0123029A984CB5
:1034A0001A400023944698460022C5E680224B46E7
:1034B000120313420AD05B46134206D11A43120389
:1034C000120BAC4688468E4CB6E64B461A431203A6
:1034D000120BBC468A4CAFE603005A46283B9A4082
:1034E00000239146984657E6584601F04BF92030A4
:1034F00040E603005246283B9A400021934677E677
:1035000001F040F920305FE6884500D2C7E64B461F
:10351000DE075D0843465B081E434346DB079A46C9
:10352000C2E60025924500D333E7039E5946B446D0
:10353000E244B245AD416D424544EB18013998452E
:1035400007D2984200D97FE000D1BCE01D1A8B461B
:103550001FE79845FAD1039D5545F2D943468B465E
:103560001D1A16E79B46CAE61500E7E65A46C90843
:1035700052070A435B0590465C0D5A4601230299A7
:1035800052021940120B8C4656E6002B00D16FE711
:1035900046444A1EB04529D91100864200D065E74D
:1035A000039A934200D061E762E70121494201207A
:1035B000C21A382A21DD029B03409C4638E60F22BE
:1035C0000A40042A00D15BE70A00111D9142924192
:1035D0005242934454E7474BE318002BE5DD0122A8
:1035E0005242F2E71D00FAE69A461CE7B04239D88B
:1035F0006ED011003AE702933AE71F2A3CDC202301
:103600009B1A0C005846994098404B1E99415B46C6
:10361000D440D340204308431A00430709D00F2366
:103620000340042B05D00100081D88429B415B42EA
:10363000D21813023AD50123029A01241A4000231A
:10364000944698460022F7E5022149428C46039DA4
:10365000E344AC46E244AA45AD416D424544ED1811
:103660002D1A96E68A1E03994D008D4289414942E2
:103670004144761803958FE71F204042C31A5846ED
:10368000D8400300202A28D040205D46821A954069
:1036900029434A1E91411943072300220B4009D0B8
:1036A0000F2300220B400800042BBDD1010053075B
:1036B0005202120BC90819430123884602990024BB
:1036C00019408C46B8E55245BED88B46002560E6C9
:1036D000039D9D42C6D3110062E70025D8E78022F2
:1036E0005B4612031A43019B1203120B9C46884649
:1036F000034CA1E5FF030000FFFFFFFEFE070000F3
:10370000FF070000F0B54F464646D6465C00C0B500
:103710001F03DB0F9A46174B0E034D00844680466D
:10372000360B6D0DC90F91463F0B640D01209D4274
:1037300008D09C4201D0A5420BD01CBC90469946B3
:10374000A246F0BD63463343F7D1AC42F5D13A43CC
:10375000F3D10120BE42F0D1C845EED1514507D08A
:10376000002DEAD163461E433000461EB041E4E717
:103770000020E2E7FF070000F0B54546DE46574669
:103780004E46E0B51F033D0B2C4F0E034C00AB46DD
:103790005D008446360B640DC90F90466D0DDB0F3E
:1037A000BC422AD0254FBD422DD0002C0FD1304332
:1037B0000700814678427841C0B2002D17D15F469C
:1037C0003A4314D14B460020002B0AD006E0002DCE
:1037D00002D15846024301D0994218D048420121F3
:1037E00008433CBC90469946A246AB46F0BD002833
:1037F000F2D00120013B1843F3E737000743D1D053
:1038000002204042EDE75F461743CED0F8E7AC42D6
:10381000E4DC03DA481E01210843E2E75E45DDD817
:1038200006D000205E45DCD20123481E1843D8E7AD
:10383000C445D3D80020C445F6D3D2E7FF07000023
:10384000F0B54E464546DE4657465C00E0B51F03E0
:10385000DB0F99462A4B0E034D00C90F8446360BE9
:103860006D0D8B4690463F0B640D9D4220D0244B3E
:103870009C4222D0002D12D1304343424341DBB25F
:10388000002C1FD0002B0CD04B460120013B0343E2
:1038900018003CBC90469946A246AB46F0BD002CB1
:1038A00016D0CB4517D05B46594201230B43EFE7B7
:1038B000310002230143EBD1D9E739000223114340
:1038C000E6D1D7E73A43DDD100230028E0D0EAE78C
:1038D0003A43E6D1E7E7A542E5DC05DBBE42E2D8A4
:1038E00007D00023BE42D3D25946012301390B43EE
:1038F000CEE7C445D7D80023C445F5D3C8E7C046B2
:10390000FF070000F0B557464546DE464E46E0B597
:103910000C0398464E00230B87B0070092469B4647
:10392000760DCD0F002E6BD06D4B9E4235D080248E
:103930005B46420F2404DB0014431C43C30099463A
:10394000684BA3469C4600230027664402934346E7
:103950001C035A00DB0F5046240B520D984600D131
:1039600076E05F4B9A426DD08023410F1B040B43DE
:103970005C49E4008C461C43C3000020624441467D
:10398000B6186940721C0191944607430F2F00D965
:10399000B0E0554ABF00D25997465B46034399466B
:1039A00000D087E000239B46023308270293CEE72E
:1039B00042460192022867D0032800D10EE2012876
:1039C00000D062E1002300240022994601990140C1
:1039D000CDB2002112030B0D120B1B051343434AFA
:1039E000240513401C436400ED0764082C4348463B
:1039F000210007B03CBC90469946A246AB46F0BDBC
:103A0000034399464FD05B46002B00D189E15846CD
:103A100000F0B8FE03000B3B1C2B00DD7AE11D22F9
:103A2000D31A3A0001005C46DA4008398C40130092
:103A30008F4023439B46B94600232D4E0027361A5C
:103A4000029384E7534623432AD10024022096E7B9
:103A50005346234320D0002C00D157E1200000F032
:103A600091FE03000B3B1C2B00DD49E11D21CB1A0D
:103A700051460200D9405346083A944093400C43C3
:103A80001B4A121A00207AE70125019B144C1D40A5
:103A90000023002299469CE70024002201206EE7C3
:103AA000534603206BE700239B460133042700267F
:103AB00002934CE7032381460C27029347E78022B9
:103AC0000023002512039946054C82E75C464B46CD
:103AD00002986FE75C464B46019502986AE7C0463C
:103AE000FF07000001FCFFFF5C5A0000FFFF0F8092
:103AF0000DFCFFFF4A464946170C1A0C1B041B0C11
:103B000008041900000C41431500884619007D4344
:103B10007943039589462900150045434D44029594
:103B200045462D0CAA46029D5544A94506D98A460C
:103B3000802149028946CA4451460391290C0491C7
:103B4000414609042D04090C88462900250C24044B
:103B50004144240C059121004143884621007943CA
:103B60008A466843414650448146080C48446F43A6
:103B7000824503D98021490289464F44010C894678
:103B800039004944029141460F0404993F0C88468C
:103B90000004C01980444146049159460F0C0904A1
:103BA000090C884659438A463900514389464146A3
:103BB0004A435146090C8B467B43D2185A449342E0
:103BC00003D980235B029B46D94451460904090C62
:103BD0008A46414661437C43130C12044B445244D1
:103BE000A1468A463C0041466C434D4351464D44F4
:103BF0000F0C7D19A94503D9802149028846444408
:103C0000049F0399B84641448B4683458041414215
:103C10008846514608042F04000C3F185846029964
:103C200010188946904292414F44BA4652429946F2
:103C30009346C244D144CB448F42BF41C2458941DF
:103C400099459B41934592417F4249422D0C5242F6
:103C50000F435B4213437F19FF185B463C19DB0D92
:103C6000059A64021C43430213435D1EAB415A464E
:103C7000C00D034352021343E20156D501205A08F6
:103C800003401343E207134364085A486044002882
:103C90004DDD5A0709D00F221A40042A05D01A1DFB
:103CA0009A429B415B42E4181300E20104D5802054
:103CB000514AC00014406044504A904200DDE3E69F
:103CC0000125DB0862071A436402019B9146220B1F
:103CD0004405640D1D407CE68022594612031142C2
:103CE00008D0144206D122431203120B45469946CE
:103CF000434C6EE65B461A431203120B404C68E6D7
:103D000003005446283B9C400023B9E600F03AFDEE
:103D10002030A6E60300283B9F400023BB4699467F
:103D20008AE600F02FFD203074E6B446ADE70125A9
:103D30002A1A382A06DD019B00241D400023002298
:103D4000994646E61F2A21DC20252000AD1A1E00D8
:103D5000AB40A840D6405D1EAB4130431843D44031
:103D6000430709D00F230340042B05D00300181D7F
:103D700098429B415B42E418230221D50125019B17
:103D800001241D4000230022994622E61F25210020
:103D90006D42281AC1400800202A1DD05F35AA1A9A
:103DA000944023435C1EA341072503431D4000228A
:103DB000002D09D00F2200241A401800042AD6D161
:103DC000030065076402220BDB082B43012599469B
:103DD000019B00241D40FCE50024E2E78022012530
:103DE0001203224301991203120B0D409946044C11
:103DF000EFE5C046FF030000FFFFFFFEFE070000E7
:103E0000FF070000F0B54646D6464F460C03C0B546
:103E1000CD0F4E00610A440F0C43C1005800400D05
:103E200084468A460F001903500F490A0143C648C9
:103E3000760DA846DB0FD200844500D1D8E00120E2
:103E40004340AB4200D1A6E06046351A002D00DCAD
:103E500005E1002810D10B00134300D1D7E06B1E01
:103E6000002B00D04BE153469F1ABA458041641A9B
:103E70004042241A01261EE0B34B9E4248D08023C4
:103E80001B041943382D00DD19E11F2D00DD4CE125
:103E900020230F005B1B10009A409F40E840531EF8
:103EA0009A41E940074317435346DF1B611ABA455D
:103EB000A44164420C1B230200D4C5E06402650ADD
:103EC000002D00D1F6E0280000F05CFC0300083B68
:103ED0001F2B00DDE9E020223C00D21A9D40D44097
:103EE0009F4025439E4200DDDBE09E1B731C1F2B81
:103EF00000DD0AE120223800D21A290097402C0068
:103F00009140D8407A1E9741DC40002601430F4380
:103F10007B0709D00F233B40042B05D03B1DBB4240
:103F2000BF417F42E4191F00230225D5864B01368D
:103F30009E4200D1AFE0854B01251C4043466207FD
:103F4000FF08640276051743240B760D1D400021FF
:103F50002403230B0C0D7E4A24051C431440330517
:103F600023435B00ED075B082B43380019001CBCA2
:103F700090469946A246F0BD012543466207FF08D8
:103F80001743E4081D40704B9E4236D0240376054B
:103F9000240B760DDBE76346F31A002B00DC94E07C
:103FA0006046002835D068488642B1D080273F045B
:103FB0003943382B00DCFDE00A43170000217A1E4C
:103FC0009741574457458041091944420C1923022F
:103FD0003AD55D4B01369E4200D14BE101225B4B4D
:103FE0001C407B0817401F43E207174364088FE714
:103FF0000800104300D024E721E723003B4300D111
:10400000B9E18022120314432403240B9FE72E00FE
:104010007EE70800104300D1CAE0581E84460028FD
:1040200000D0E7E0524452458041641840422418D1
:1040300017000126230207D50226CFE764462C434A
:1040400000D1B3E12C0067467B0700D062E763072D
:10405000FF081F4301254346E4081D4093E7002D58
:1040600078D1751C6D056D0D012D00DCF2E0504618
:10407000801A8245BF41651A7F42ED1B84462802A3
:1040800000D48CE05046171ABA4292410C1B55429C
:10409000651B984614E70125434600241D40002770
:1040A00055E72A4CF61A2C4032E73D002838854067
:1040B000002717E7380000F065FB203006E70A43C9
:1040C000170000217A1E9741EEE6002B00D0E5E0B4
:1040D000731C9C465B055B0D012B00DC9FE01A4BBB
:1040E0009C4500D1C5E0524452458041641840428D
:1040F0002418E707520817436408664608E7124881
:10410000854200D185E01D00BCE629001F3EF1403C
:10411000202B00D17FE04022D31A9D402F437D1EEB
:10412000AF4100240F4300268EE72B000F00203BF9
:10413000DF40202D71D040235D1BA9400A43511E52
:104140008A4100211743AFE6FF070000FFFF7FFF12
:10415000FFFF0F80002E3ED0B34EB44545D08026E1
:1041600036046D423443382D00DDA8E01F2D00DDFC
:104170001FE1202627005046761BB740E840074342
:104180005046B040461EB041EC403843171ABA4280
:1041900092410C1B5242A41A664698468BE664462E
:1041A00067462C4300D08BE6002500260027EAE670
:1041B0001E00ADE61F2B60DC2027F81A0F00844696
:1041C00087401000D840074360468240501E82411D
:1041D000D9401743F5E626005046064305D0ED4387
:1041E000002DD3D0904EB445BDD10C0017006646CB
:1041F00098468DE68C4883420BD06346D9E6002D65
:1042000000D096E00800104300D1E2E00C00170057
:104210009846854E7CE6002580E700218EE7230046
:1042200050460343002E00D0A8E0002B00D1DEE072
:104230000B00134300D16BE6524452458041641891
:10424000404224181700230200D4FDE6774B66464F
:104250001C405DE6250050460543002ECFD1002DC1
:104260004FD10C00144300D1A0E00C001700984679
:104270004EE666460024002785E61F000800203F22
:10428000F8400700202B00D18EE04020C31A99404F
:104290000A43511E8A410021174392E6002E14D191
:1042A00026005046064362D0DB43002B5CD18718C2
:1042B0009742924164185242A418664687E65046D7
:1042C0002043441EA041002460E7574EB4454ED021
:1042D000802636045B423443382B00DD7FE01F2B01
:1042E00000DD8BE0202627005046F61AB740D84064
:1042F00007435046B040461EB0410743DC40BF185C
:10430000D6E70D00154300D102E65046801A8245DB
:10431000BF41651A7F42ED1B8446280200D48DE61A
:104320005046171ABA4292410C1B5242A41A9846A0
:10433000EEE50D00154300D16BE750466707C00856
:1043400007438020E4080003044207D0CD0805425B
:1043500004D12C009846D70849070F437B0FE4008F
:104360001C43FF00304ED3E52F4EB445B4D10C00B2
:1043700017006646CCE500270024E8E5002B39D07D
:104380000B00134300D144E7C008670707438020B0
:10439000E40800030442E1D0CB080342DED1D70891
:1043A00049070F431C00D9E7002171E700250027CA
:1043B000E9E52E002700203EF740202D2FD0402693
:1043C000751BAC4050462043441EA0410024384396
:1043D000DCE6802400252403134E0027D3E5504655
:1043E00020430700781E87410024BF1860E70C00B7
:1043F00017008DE50C0017000B4E89E51E00270005
:10440000203EF740202B0CD04026F31A9C4050460B
:104410002043441EA04107430024BF1848E700245E
:10442000D0E70024F3E7C046FF070000FFFF7FFF4F
:1044300070B50E4E0D031C0349005B002D0B490D9A
:10444000240B5B0DB14204D0084900208B4208D0F8
:1044500070BD05430120002DFAD1044900208B4294
:10446000F6D114432000441EA041F1E7FF070000ED
:1044700030B5134D0A034B00120B5B0DC90F00241E
:10448000AB4210DD0F4CA3420FDC80240E4D6403C1
:104490002243ED1A1F2D0BDD0C48C31ADA4054429B
:1044A000002900D11400200030BD094BCC18FAE7D8
:1044B000084CE840A44663449A400243EFE7C046F4
:1044C000FE0300001D04000033040000130400007C
:1044D000FFFFFF7FEDFBFFFF70B5002830D0C31753
:1044E000C4185C40C50F200000F04CF9174B184A67
:1044F0001B1AD21A1F2A18DD164AD21A944000221B
:1045000024035B05240B5B0D0021100024030A0D1E
:10451000240B12052243104C1B05224013435B0061
:10452000ED075B082B43190070BD210091400A0084
:104530000B21081AC4405B052403240B5B0DE3E741
:104540000025002300240022DEE7C0461E040000F0
:104550003304000013040000FFFF0F8010B5041E99
:1045600028D000F00FF9154B154A1B1AD21A1F2A32
:1045700015DD144AD21A9440002224035B05240B53
:104580005B0D0021100024030A0D240B12052243A9
:104590000D4C1B05224013435B00590810BD210040
:1045A00091400A000B21081AC4405B052403240B28
:1045B0005B0DE6E7002300240022E2E71E04000072
:1045C0003304000013040000FFFF0F804100090EB8
:1045D0004B1C70B5DBB24602750AC40F012B14DD0B
:1045E000E0239B006D07360BCB1800210A0D280035
:1045F00012051C4D32435B052A405B0813435B00E8
:10460000E4075B082343190070BD002914D1002D75
:104610001ED0280000F0B6F80A281CDC0B232A0064
:104620001B1ADA40030015339D400F4B12031B1A6F
:104630005B05160B5B0DD8E7002D06D0320B8026EC
:1046400036036D071643094BCFE7084B0026CCE72E
:1046500000230026C9E703002A000B3B9A400025EF
:10466000E3E7C046FFFF0F8089030000FF0700005B
:10467000F0B54C00640D0B03621C450F5B0A52053C
:104680002B43C90FC500520D012A28DD3A4AA6184E
:10469000FE2E1BDC002E3EDD80010200501E8241FA
:1046A0006D0F2A43DB0013435A0704D00F221A4030
:1046B000042A00D004338022D2041A405AD0013692
:1046C000FF2E03D09B015B0AF4B201E0FF2400231C
:1046D0005802E405400AC90720430843F0BD002CF6
:1046E00007D01D43F2D08020DB0080040343FF2667
:1046F000DAE72B4303D00523DB08FF2C03D05B0252
:104700005B0AE4B2E4E7002B32D08020C00303430D
:104710005B025B0ADCE73200173214DB80221E27C3
:1047200012041343BF1B1F2F0FDC144A944664442A
:104730002A00A5402E00A340751EAE41FA40334327
:1047400013430026B0E70024D5E702225242961B0D
:104750001A00F240202F09D0094884466444A3403F
:104760002B435D1EAB41002613439DE70023F7E773
:104770000023ADE73400BFE780FCFFFF82FCFFFFB2
:10478000A2FCFFFF1C2101231B04984201D3000C53
:1047900010391B0A984201D3000A08391B099842B4
:1047A00001D30009043902A2105C40187047C046CA
:1047B00004030202010101010000000000000000EA
:1047C000014B18687047C0461800002070B50026DD
:1047D0000C4D0D4C641BA410A64209D1002601F01B
:1047E000A9F90A4D0A4C641BA410A64205D170BD5C
:1047F000B300EB5898470136EEE7B300EB58984703
:104800000136F2E7405B0000405B0000405B0000C7
:10481000445B0000002310B59A4200D110BDCC5C6F
:10482000C4540133F8E703008218934200D1704763
:1048300019700133F9E700000FB40B4B13B51C6876
:10484000002C05D0A369002B02D1200000F0F2FA61
:1048500005AB049AA1682000019300F0C7FC16BCC8
:1048600008BC04B01847C0461800002070B5050009
:104870000E00002804D08369002B01D100F0DAFA81
:10488000AB69AC68002B02D1280000F0D3FA244BAE
:104890009C420FD16C68A3891B0702D52369002BAA
:1048A00020D12100280000F057F900281AD001205B
:1048B000404270BD1B4B9C4201D1AC68EBE71A4BE8
:1048C0009C42E8D1EC68E6E7013B0136A360002B8F
:1048D00004DAA269934216DB0A2914D023685A1C11
:1048E000226019703178A3680029EDD1013BA360E3
:1048F000002B0FDA22000A31280000F0D7F8431C01
:10490000D5D00A20D5E72200280000F0CFF8431CBC
:10491000E8D1CCE70A2023685A1C22601870C8E747
:10492000C05A0000E05A0000A05A000010B5034B26
:1049300001001868FFF79AFF10BDC046180000205C
:104940004A424A41802310B55200DB0000F002F8D1
:1049500010BD0000F0B51D004F4B85B01E6804006F
:104960000F000092002E05D0B369002B02D1300059
:1049700000F060FA494B9C4250D17468009B022BB6
:1049800005D0012B00D984E0002D00DA81E0210060
:10499000300000F0E1F9616B002908D023004433B6
:1049A000994202D0300000F051FB002363630023E2
:1049B000A3616360A3891B0603D52169300000F061
:1049C00045FBA389364A1340A381009B022B5AD092
:1049D00003AB02AA2100300000F0C2FAA3891843F9
:1049E000A081002D24D1029D280000F025FB019517
:1049F000071E42D1029B0193AB4239D101204042B4
:104A00000223A2891343A3810023A3602300473319
:104A1000236023610123636105B0F0BD214B9C42FB
:104A200001D1B468AAE7204B9C42A7D1F468A5E75E
:104A3000002FD9D0B369002B02D1300000F0FAF971
:104A4000009B012B03D1A389009A1A43A28108205D
:104A5000A389276027616561184018D0012018409C
:104A60000023984211D06D42A360A5611800D3E7DE
:104A7000019800F0E1FA071EC0D08023A289019DB1
:104A80001343A381D6E70020BAE7A560C4E7A0607E
:104A9000C2E701204042BFE718000020C05A0000D2
:104AA0005CF3FFFFE05A0000A05A0000F8B50500D3
:104AB0000E001400002804D08369002B01D100F0FF
:104AC000B9F9224B9C422DD16C68A369A360A389DC
:104AD0001B0731D52369002B2ED023682269F7B23A
:104AE000981A6369F6B2984205DB2100280000F0AD
:104AF00033F9002826D1A3680130013BA360236865
:104B00005A1C22601F706369984204D0A389DB0796
:104B10001AD50A2E18D12100280000F01DF900280E
:104B200012D00FE00A4B9C4201D1AC68CDE7094B93
:104B30009C42CAD1EC68C8E72100280000F00CF8BC
:104B40000028CAD0012676423000F8BDC05A0000C5
:104B5000E05A0000A05A0000364B70B51D680600F0
:104B60000C00002D05D0AB69002B02D1280000F00D
:104B700061F9314B9C420FD16C680C23E25E93B219
:104B800019072DD4D90611D40923012033603733F6
:104B90001343A381404270BD284B9C4201D1AC68B5
:104BA000EBE7274B9C42E8D1EC68E6E75B0713D5BF
:104BB000616B002908D023004433994202D03000B1
:104BC00000F044FA002363632422A3899343A38162
:104BD00000236360236923600823A2891343A38110
:104BE0002369002B0BD1A0218022A3898900920088
:104BF0000B40934203D02100300000F0D9F901238B
:104C0000A289134011D00023A36063695B42A361B2
:104C1000002023698342BED10C23E25E1306BAD57D
:104C200040231343A3810138B5E7920700D4636999
:104C3000A360EDE718000020C05A0000E05A000011
:104C4000A05A0000F7B58A8905000C00130760D44C
:104C50004B68002B04DC0B6C002B01DC0020FEBD3C
:104C6000E76A002FFAD000232E682B6080235B01B7
:104C70001A4034D0606DA3895B0706D56368C01AFB
:104C8000636B002B01D0236CC01A0200216A002341
:104C90002800E76AB847A189431C06D12B681D2B61
:104CA00031D82C4ADA40D3072DD50023636023691D
:104CB0002360CB0405D5431C02D12B68002B00D107
:104CC0006065616B2E600029C8D02300443399428F
:104CD00002D0280000F0BAF900206063BFE701238A
:104CE000216A2800B847431CC5D12B68002BC2D0CD
:104CF0001D2B01D0162B01D12E60AFE74023A289D6
:104D00001343A381ABE740230B430120A38140421F
:104D1000A5E70F69002FA1D00B680F60DB1B019383
:104D20000023920700D14B69A360019B002B00DC9C
:104D300094E7019B3A00216A2800A66AB047002840
:104D400003DC4023A2891343DFE7019B3F181B1AB2
:104D50000193EAE7010040200B6970B505000C00E3
:104D6000002B01D1002070BD002804D08369002BE6
:104D700001D100F05FF80B4B9C4209D16C680C220A
:104D8000A35E002BEED021002800FFF75BFFEAE7CF
:104D9000054B9C4201D1AC68F1E7044B9C42EED13B
:104DA000EC68ECE7C05A0000E05A0000A05A00008E
:104DB00010B5024900F0B2F810BDC046594D0000D0
:104DC000002310B504000360436083608181436663
:104DD000C281036143618361190008225C30FFF7DF
:104DE00022FD054B24626362044BA362044BE36221
:104DF000044B236310BDC046595700008157000083
:104E0000B9570000E557000070B568254A1E5543A4
:104E10000E002900743100F063F9041E08D000214F
:104E20002A00016046600C30A0606832FFF7FBFC8E
:104E3000200070BD836913B50400002B28D1836462
:104E4000C3640365134B144A1B6882620193984242
:104E500001D101238361200000F020F86060200070
:104E600000F01CF8A060200000F018F80022E060BC
:104E700004216068FFF7A4FF01220921A068FFF761
:104E80009FFF02221221E068FFF79AFF0123A3612E
:104E900013BDC0469C5A0000B14D0000F8B51E4B32
:104EA00007001E68B369002B02D13000FFF7C2FF74
:104EB0004836B4687368013B04D53368002B07D0CB
:104EC0003668F6E70C22A55E002D0DD06834F2E7B7
:104ED00004213800FFF798FF30600028F0D10C2340
:104EE00004003B602000F8BD012320005B42E38109
:104EF0000233A38165662560A560656025616561F3
:104F0000A561082229005C30FFF78DFC6563A5636D
:104F1000A564E564E6E7C0469C5A0000F7B50400C6
:104F20000700002601914834002C01D13000FEBD5D
:104F30006368A5680093009B013B009301D524683A
:104F4000F2E7AB89012B08D90E22AB5E013304D006
:104F500029003800019B984706436835EBE70000BD
:104F600070B50E001D000E23C95E90B0140000291C
:104F700007DA00232B60B3891B0611D48023DB00E2
:104F80000FE001AA00F05AFC0028F2DBF022029B9D
:104F900012021340054A9B185A4253412B60EDE719
:104FA00040230020236010B070BDC04600E0FFFF2A
:104FB000F7B502268B8905000C00334206D023008A
:104FC00047332360236101236361F7BD01AB6A4668
:104FD000FFF7C6FF00990700280000F081F80028BD
:104FE00008D10C22A35E9A05EFD4032293431E43FB
:104FF000A681E4E70F4BAB628023A28920601343B4
:10500000A381009B20616361019B002B0DD00E23C7
:10501000E15E280000F024FC002806D00322A389CA
:1050200093431A0001231343A381A0893843A0812D
:10503000CBE7C046B14D000010B5034B0100186826
:1050400000F04EF810BDC0461800002070B50500F5
:10505000002910D00C1F2368002B00DAE418280068
:1050600000F02FFC1D4A1368002B05D1636014600B
:10507000280000F027FC70BDA34209D92168601800
:105080008342F3D118685B6841182160EEE7130092
:105090005A68002A01D0A242F9D919685818A042CA
:1050A0000BD120680918581819608242E0D11068A5
:1050B0005268411819605A60DAE7A04202D90C23FD
:1050C0002B60D5E721686018824203D110685268CE
:1050D0004118216062605C60CAE7C046CC010020D4
:1050E000032370B5CD1C9D43083506000C2D1ED240
:1050F0000C25A9421DD8300000F0E3FB254A1468B6
:105100002100002919D1244C2368002B03D1300041
:1051100000F010FB20602900300000F00BFB431C66
:105120002CD10C233000336000F0CCFB03E0002DC9
:10513000DFDA0C233360002070BD0B685B1B1AD4D0
:105140000B2B03D90B60CC18256003E08C420ED1E9
:1051500063681360300000F0B5FB200007220B30BD
:10516000231D9043C31AE7D05A42E250E4E74B684C
:1051700063600C00EEE70C004968C2E70323C41C1F
:105180009C43A042E0D0211A300000F0D3FA431C27
:10519000DAD1C6E7CC010020D0010020936810B519
:1051A000013B9360002B05DA9469A34208DBCBB284
:1051B0000A2B05D01368581C10601970C8B210BDB6
:1051C000FFF774FCFBE7F8B506000F001400D518D4
:1051D000AC4201D1002007E021783A003000FFF70F
:1051E000DDFF0134431CF3D1F8BD0000F0B59FB0E2
:1051F00006000F0014000593002804D08369002BDB
:1052000001D1FFF717FE7F4B9F425CD17768BB89C6
:105210001B0762D53B69002B5FD0002306AD6B6195
:1052200020336B761033AB760294029C2378002BEC
:105230005DD1029BE31A04930DD0049B029A3900BE
:105240003000FFF7C0FF431C00D1CCE06A69049B2B
:10525000944663446B612378002B00D1C3E00122A4
:10526000002352426A6002A95432521801342B6062
:10527000EB60AB601370AB6521780522624800F0EB
:1052800015FB631C9C46002835D12968CB0604D544
:10529000532302AA20309B1818700B0704D5532300
:1052A0002B2002AA9B18187023782A2B2CD00020C0
:1052B0000A21099B2278303A092A00D86BE000289D
:1052C0002AD0099328E0514B9F4201D1B7689EE74D
:1052D0004F4B9F429BD1F76899E739003000FFF7A9
:1052E0003BFC002899D0012040421FB0F0BD252B87
:1052F0009FD001349AE7444B2968C01A01238340A8
:105300000B432B606446B7E7059B181D1B6805908F
:10531000002B3ADB0993644623782E2B0BD163785C
:10532000621C2A2B3FD1059B02341A1D1B68059273
:10533000002B35DB079321780322364800F0B6FABC
:10534000002807D0334B2A68C01A402383401343F8
:105350002B6001342178631C06222F4802932976A2
:1053600000F0A4FA002844D02C4B002B2FD1296840
:10537000059B0722C90528D59B189343083305933D
:105380006B69039A9B186B614FE75B42EB600223EA
:105390000B432B60BFE74B4301349B18012089E787
:1053A00001235B42C6E7002314000A201A006B6049
:1053B00021783039092903D9002BBCD00792BAE7EC
:1053C0004243013452180123F2E70733D5E705AB16
:1053D00000933A00124B2900300000E000BF039018
:1053E000039B0133CCD1BB895B0600D57BE70B98CF
:1053F0007BE705AB00933A00094B2900300000F031
:105400007FF8ECE7C05A0000005B0000E05A0000A3
:10541000A05A0000065B00000A5B000000000000CC
:10542000C7510000F7B5150001938A680B69009019
:105430000C00934200DA130022002B6043321278F2
:10544000002A01D001332B6023689B0602D52B680C
:1054500002332B60062723681F4027D023004333E5
:105460001B785A1E93412268920630D4220001997B
:1054700043320098089EB047431C25D0062320687D
:105480002A68E16803400025042B03D18D1AEB4301
:10549000DB171D40A3682269934201DD9B1AED18BA
:1054A0000027BD4220D1002010E00137E3682A68C0
:1054B0009B1A9F42D2DA22000123193201990098E7
:1054C000089EB047431CF0D101204042FEBD302071
:1054D000E1184331087021005A1C45310978A2189F
:1054E000433202331170C1E7220001231A320199BD
:1054F0000098089EB047431CE6D00137D1E7000072
:10550000F0B58BB006920A004332079305900492DF
:105510000A7E0C00109B6E2A00D18FE017D8632AF8
:105520002CD008D8002A00D199E0582A54D026005F
:105530004236327029E0642A01D0692AF7D1216805
:105540001A68080623D5111D1960156825E0732A0D
:1055500000D188E008D86F2A29D0702AE7D120220C
:1055600009680A43226003E0752A20D0782ADED138
:1055700022007821453211706C4A30E00E001A6822
:105580004236111D196013683370012379E0490612
:10559000D9D5111D19600023D55E002D03DA2D2306
:1055A000049A6D421370624B0A2703932FE0206820
:1055B0001968050603D5081D18600D6805E040064A
:1055C000F9D50D68081D1860ADB2594B0827039333
:1055D0006F2A18D00A2716E045310A70544A039200
:1055E0001A682168101D18601568080622D5CB07B7
:1055F00002D52023194321601027002D03D1202339
:1056000022689A4322602300002243331A706368A1
:10561000A360002B5CDB0422216891432160002DF4
:1056200058D1049E002B64D02600039B42361B7881
:1056300033705EE04806DAD5ADB2D8E709681A687B
:10564000080605D5111D1960136862691A6006E025
:105650004906F7D5111D19601368A28A1A80002324
:10566000049E236154E01A68111D19601668002118
:105670006268300000F01AF9002801D0801B6060D9
:10568000636823610023049A137041E023693200A8
:1056900006990598079DA847431C43D02368002519
:1056A0009B070FD4099BE06898423DDA18003BE065
:1056B00022000123193206990598079EB047431C22
:1056C00030D00135E368099A9B1A9D42F0DBE9E787
:1056D000002DA9D0049E28003900FCF7C5FD039BCE
:1056E000013E5B5C280033703900FCF737FD051E76
:1056F000F1D1082F09D12368DB0706D56368226939
:10570000934202DC3023013E3370049B9B1B2361D8
:10571000079B09AA00932100069B0598FFF782FECC
:10572000431CB3D1012040420BB0F0BD225B00000E
:10573000115B0000002370B5064C050008002360D3
:10574000FCF77CF9431C03D12368002B00D02B60AD
:1057500070BDC0469C02002070B50C000E25495F4C
:1057600000F0B2F8002803DB636D1B18636570BDA1
:10577000A389024A1340A381F9E7C046FFEFFFFF68
:10578000F8B51F008B8905000C001600DB0505D558
:105790000E23C95E0022022300F074F8A389054A93
:1057A00028001340A38132000E23E15E3B0000F08D
:1057B0001FF8F8BDFFEFFFFF70B50C000E25495F25
:1057C00000F060F8A389421C03D1054A1340A3816D
:1057D00070BD802252011343A3816065F8E7C04683
:1057E000FFEFFFFF10B50E23C95E00F015F810BDE6
:1057F00070B50500080011000022064C22601A0056
:10580000FBF770F9431C03D12368002B00D02B60F9
:1058100070BDC0469C020020002370B5064C0500F8
:1058200008002360FCF71AF9431C03D12368002BFE
:1058300000D02B6070BDC0469C020020002370B5D4
:10584000064C0500080011002360FCF70AF9431C10
:1058500003D12368002B00D02B6070BD9C02002078
:10586000002370B5064C050008002360FCF7FEF825
:10587000431C03D12368002B00D02B6070BDC046B1
:105880009C02002070B50500080011000022064CA3
:1058900022601A00FCF7ECF8431C03D12368002BAC
:1058A00000D02B6070BDC0469C020020C9B2821897
:1058B000904201D10020704703788B42FBD0013029
:1058C000F6E770477047000070B50500080011004A
:1058D0000022064C22601A00FBF7E8F8431C03D1B3
:1058E0002368002B00D02B6070BDC0469C020020B6
:1058F0000200000003000000280000002900000052
:105900000400000005000000060000000700000081
:105910002000000021000000220000002300000001
:1059200024000000250000002600000027000000E1
:1059300008000000090000000A0000000B00000041
:1059400000080042000C0042001000420014004217
:1059500000180042001C004225635B324A002563A8
:105960005B7500202D2D1B5B33313B316D20506565
:105970006E6775696E27731B5B303B3B34306D205F
:1059800053414D443231204144432044656D6F20E2
:105990007573696E6720444D41202D2D200D0056F2
:1059A0006F6C746167653A2025642E253033640975
:1059B0000054656D70657261747572653A20256476
:1059C0002E253033640025635B324B0025635B3149
:1059D000420000006C6F670000000000C42400005B
:1059E000142400001424000012240000B624000037
:1059F000B6240000AC24000012240000B6240000ED
:105A0000AC240000B624000012240000BC240000D6
:105A1000BC240000BC2400004C250000943200008F
:105A200076320000303200004E310000303200008B
:105A300068320000303200004E3100007632000043
:105A400076320000683200004E310000463100001E
:105A50004631000046310000AC340000F43A00004A
:105A6000B4390000B4390000B0390000CC3A00006D
:105A7000CC3A0000BE3A0000B0390000CC3A000039
:105A8000BE3A0000CC3A0000B0390000D43A000021
:105A9000D43A0000D43A0000D83C00001C0000209A
:105AA00000000000000000000000000000000000F6
:105AB00000000000000000000000000000000000E6
:105AC00000000000000000000000000000000000D6
:105AD00000000000000000000000000000000000C6
:105AE00000000000000000000000000000000000B6
:105AF00000000000000000000000000000000000A6
:105B0000232D302B2000686C4C00656667454647A6
:105B10000030313233343536373839414243444529
:105B20004600303132333435363738396162636498
:105B300065660000F8B5C046F8BC08BC9E467047D4
:105B4000DD000000F8B5C046F8BC08BC9E467047B2
:045B5000B50000009C
:105B5400000000000000000005000000401F0000DD
:105B640008000000010100001C00002000000000EB
:105B7400C05A0000E05A0000A05A000000000000D3
:105B84000000000000000000000000000000000011
:105B94000000000000000000000000000000000001
:105BA40000000000000000000000000000000000F1
:105BB40000000000000000000000000000000000E1
:0C5BC400000000000000000000000000D5
:04000003000019815F
:00000001FF
